:020000040000FA
:040000007CEF00F0A1
:100008000782F2A60AEF00F00CEF00F07AEF00F09A
:10001800F2A011EF00F013EF00F07AEF00F0000EFD
:1000280081BE010E036E0350D8A41DEF00F01FEF30
:1000380000F079EF00F08B908B8E820E046EDE0E4E
:10004800E82EFED7042EFCD7030E066E80BA2FEFDB
:1000580000F031EF00F034EF00F00650040F066EA8
:1000680080B039EF00F03BEF00F03EEF00F00650B3
:10007800020F066E80B843EF00F045EF00F047EF3F
:1000880000F00628066E80B24CEF00F04EEF00F04C
:1000980050EF00F00604066E80B455EF00F057EFFD
:1000A80000F05AEF00F00650FE0F066E010E056EC6
:1000B80067EF00F01A0E046EF80EE82EFED7042E35
:1000C800FCD700D0052A0550065CD8B06EEF00F0CA
:1000D80070EF00F05EEF00F08B9E8B80340E046EA4
:1000E800F20EE82EFED7042EFCD7F29007921100EC
:1000F800A6EF00F0D388D38AD38CD396D350FC0BC9
:100108000109D36EF28CF28EF19EF180F290F286A4
:100118003F0E926E3F0E776E9368F00E786E800EEB
:100128007A6E7E0E946E000E7E6E000E7F6E010E4D
:10013800D16E8B808B9EF28E8B9E0400A0EF00F018
:100148007CEF00F0036A026A016A079007920001D7
:040158007EEF00F046
:020000040020DA
:08000000FFFFFFFFFFFFFFFF00
:020000040030CA
:0E000000FF281F10FF8085FF03C003E00340B0
:00000001FF
